:10000000F01F0010BD330000B9330000B933000009
:10001000B9330000B9330000B9330000000000001C
:10002000000000000000000000000000B9330000E4
:10003000B933000000000000B9330000F5120000E1
:10004000A1100000A1100000A1100000A1100000EC
:10005000A1100000A1100000A1100000A1100000DC
:10006000A1100000A1100000A1100000A1100000CC
:10007000A1100000B5330000B5330000B533000017
:10008000AD130000C5130000DD130000F5130000E0
:10009000B5330000D5140000B5330000B5330000BF
:1000A000B5330000B5330000B5330000B5330000B0
:1000B000B5330000B5330000B5330000B5330000A0
:1000C00008B500230B60036000F068FD08BD08B5AB
:1000D0000A20002101F00AF908BD000038B50C4BD8
:1000E0000D1C041C19680B4803F09CF9212103F036
:1000F00099F9011C012001F0A9F9012001F086F90C
:10010000291C201C02F0E8FC012001F08FF938BD09
:1001100078800440001BB70008B50A4B0A481968EC
:1001200003F080F9212103F07DF9011C012001F089
:100130008DF9012001F06AF902F0ACFC012001F018
:1001400075F908BD78800440001BB70013B59620F0
:10015000000201F0FDF918480D210C2200F0FEFB11
:1001600000F03CFB15480021032200F06BFC00F07E
:100170003FFBFFF7D1FF1248124901F0D1FB0024E9
:1001800001F090FA002802D000F0B2FE00240A200C
:1001900001F0DCF8684601A9FFF792FF009B002BF5
:1001A00003D1094B01349C42EADDFFF7B5FF074854
:1001B00001F0B6FB13BDC046DD370000EC35000092
:1001C000FB350000063600006F1700000D360000FA
:1001D00073B518200021FFF781FF0024384E01205D
:1001E00001F024F9374D9835002C01D0002000E0B3
:1001F0000620012101F07AF8684601A9FFF760FFA7
:10020000009B002B21D1002CF0D12B68002B0DD0AE
:100210002D4B00941A6811321A6004E002F0E4FBDE
:10022000009B01330093009B102BF7DD274BF61842
:10023000DED518200021FFF751FF224B94331C68B4
:1002400063425C4100F09EFACEE7002C03D0182BED
:10025000C5D100F0D5FA009B182B10D1019BC22B01
:1002600029D11B4B0022196801311960022900D1E4
:100270001A6001921FE0FFF769FF00230193154BFD
:100280001548196803F0CEF8212103F0CBF8011CC2
:10029000012001F0DBF8012001F0B8F80098019985
:1002A00002F01AFC074B94331B68002B95D100F029
:1002B00069FA012492E7019B732BE0D1DBE7C0468A
:1002C00020BF020088040010C00200100CFEFFFFD7
:1002D0007001001078800440001BB70030B58BB06F
:1002E00002AC01F08BFB00F025FC00F089FA0C2237
:1002F00028480D2100F032FB00232749201C2370E1
:1003000003F04AF9254D201C291C03F045F9244926
:10031000201C03F041F9291C201C03F03DF9214960
:10032000201C03F039F900F0EFFD1F48211C01F0FB
:10033000F7FA3C2500F052FAA9B2201C032200F083
:1003400081FB013D00F054FA1E2000F0FFFF022D5A
:10035000F0D102F071FA0B23009314481E231449C4
:10036000144A02F023FB00200421012200F0E8FDE2
:100370000020021C042100F031FE00200521012292
:1003800000F0DEFD00200521021C00F027FEFFF733
:100390001FFFC046DD37000006360000A95B0000E5
:1003A0001836000020360000693600008133000056
:1003B000C1000000C002001000B500E00130037869
:1003C000202BFBD000BD00B5031C303BDAB2092A5C
:1003D00001D8181C08E020231843031C613B573840
:1003E000052B01D90120404200BD70B50E1CFFF75E
:1003F000E3FF0025041C06E0FFF7E5FF002805DB0E
:100400002D010543013420780028F5D13560201CEA
:1004100070BD000070B5054E051C0E24013C295D21
:10042000301C01F07DFA002CF8D170BD233600009D
:1004300000B50E23013BC25C002A03D1002BF9D189
:10044000012000E0002000BDF8B500240E270323A2
:100450001C4221D13E1C66432B4D7019FFF7E8FF6B
:10046000002815D0601C78434019FFF7E1FF0028F1
:100470000ED0301C1C304019FFF7DAFF002807D0DF
:100480002A367019FFF7D4FF002801D004340DE09C
:100490001E48211C01F044FA381C60431A4B0134F9
:1004A000C018FFF7B7FF1A4801F03AFAFF2CCEDD6B
:1004B000184801F035FA184C201CFFF7ABFF174D18
:1004C0004221281C01F02CFA201C0E30FFF7A2FF5D
:1004D0004321281C01F024FA201C1C30FFF79AFF4E
:1004E0000F4801F01DFA201C2A30FFF793FF281C4B
:1004F0004E2101F015FA201C3830FFF78BFF616D9B
:10050000084801F00DFAF8BD240500102636000059
:10051000A85B00002F36000088040010353600006C
:100520003C3600004236000070B50E1CFFF744FF59
:100530000D25041C2078FFF746FF002807DB013457
:100540007055013DF6D2201CFFF736FF00E0002079
:1005500070BD000073B5394D08682B78002B06D1AB
:10056000374801F0DDF902F067F9012342E0037832
:10057000412B1BD1334C0230211CFFF7D5FF002843
:1005800051D00378422B4ED1211C02300E31FFF79F
:10059000CBFF002847D00378432B44D1211C0230E5
:1005A0001C31FFF7C1FF002846D13CE04D2B23D181
:1005B000254C0230211CFFF7B7FF002833D0037809
:1005C0004E2B30D1211C02300E31FFF7ADFF002839
:1005D00029D00378472B26D1023001A9FFF705FF68
:1005E000019B002B1FDB2A3C63651848184901F06A
:1005F00097F900232B701FE001A9FFF7F6FE03789F
:10060000202B01D0002B0ED1124E00240E25019973
:10061000611869438919FFF787FF002803D0013467
:10062000042CF4D108E002F007F908480A4901F067
:1006300077F9024B00221A7073BDC0469802001071
:100640004E36000088040010B2040010643600002A
:100650006E360000240500107136000037B54C6876
:1006600024E0201CFFF7A8FE01A9FFF7BEFE019BB6
:10067000041C002B1DD0D8B2FF2B09DD00F0FCF9C3
:10068000051C01980012C0B200F0F6F9019003E0D9
:1006900000F0F2F9002501900198002802D0291CF1
:1006A000FFF71CFD23785A1E9341E4182378002B92
:1006B000D7D137BD08B5064A012113784B401370D6
:1006C00001D0044900E00449044801F029F908BDBB
:1006D000750300107836000080360000893600006F
:1006E00070B5051C01200821021C00F077FC0724CE
:1006F000012601200821002200F070FC2A1C224162
:1007000032400020022100F069FC01200821021C77
:1007100000F064FC013CECD270BD10B50021041C5B
:100720000A1C022000F05AFC201CFFF7D9FF10BD64
:10073000F7B5012300930023019372B66C46061CA3
:1007400002AF01CC50235B421843C0B2FFF7E5FF74
:100750000020FFF7E2FF1020FFF7DFFFE020FFF7A8
:10076000DCFF002502200021012200F037FC705D33
:100770000135FFF7B5FF842DF4D18436BC42E0D1BA
:1007800062B6F7BD08B5AC20FFF7C7FFAE20FFF794
:10079000C4FFA520FFF7C1FF08BD08B5AF20FFF7D4
:1007A000BCFFA420FFF7B9FF08BD08B5AE20FFF7D6
:1007B000B4FF08BD10B5041CF820FFF7AEFF201CE5
:1007C000FFF7ABFF10BD10B5041C8120FFF7A5FF9C
:1007D0003F202040FFF7A1FF10BD000008B5842294
:1007E00002480021520001F0C8F808BD7D03001046
:1007F00008B50248FFF79CFF08BDC0467D03001006
:1008000008B50120021C082100F09AFB0120021CFF
:10081000082100F0E3FB00200221012200F090FB00
:1008200000200221012200F0D9FB02200021012238
:1008300000F086FB02200021012200F0CFFB022005
:100840000621012200F07CFB02200621012200F09B
:10085000C5FB0320011C012200F072FB0320011CD8
:10086000012200F0BBFB0320011C002200F0B6FBBC
:1008700002200621002200F0B1FB06210122022005
:1008800000F0ACFBFFF7AAFFFFF7B2FFA220FFF7D3
:1008900044FFA020FFF741FFC020FFF73EFF0020EC
:1008A000FFF788FF0A2000F051FD4020FFF735FFD9
:1008B0002C20FFF732FF322000F048FD2E20FFF7FA
:1008C0002CFF322000F042FD2F20FFF726FF0A20E8
:1008D00000F03CFD2520FFF720FFAF20FFF71DFFB4
:1008E000A420FFF71AFF0020FFF76DFF08BD0000EE
:1008F00000B50F290ED883280CD8CB088422534387
:100900000722C0181140044B80220A41111C1A5CB6
:100910001143195400BDC0467D030010F0B55B18AB
:10092000DBB216E08425CC086C4307270F408025F6
:1009300004193D41EFB2A6189C4605E0064BE518A8
:100940002B7801343B432B70B442F7DB0131634613
:10095000C9B29942E6D3F0BD7D03001000B5084B43
:100960001860084B1970084B20211A70074B19703A
:10097000074BD1081970500701D00131197000BD23
:10098000780300108504001087040010860400100E
:100990007C030010F0B5284B89B01B780024C01AE6
:1009A000264B069205911B68221C04E002310C19AB
:1009B0000132A4B2D2B2195D8242F7DB1B195B7817
:1009C0000391029300222CE000994B4303999A195A
:1009D0008A4214DA194A0025126892191219D3189A
:1009E0009B7804930123049AAB40134204D07919F5
:1009F000C9B20798FFF77CFF0135082DF2D1013607
:100A00000837F6B2FFB206E00099059A069F8B18E8
:100A1000DBB2002607930A490B789E42D4D3019A91
:100A2000013201926B461B79029900938B42EBD302
:100A300009B0081CF0BDC046860400107803001001
:100A40007C030010F7B5171C061C0D1C00F0B5FF49
:100A500080B201900024FFB208E0305DE9B23A1C98
:100A6000FFF798FF01302D18ADB20134019AA3B2FF
:100A70009342F2D3F7BD000000B50F2302091840DE
:100A80008000031F00D52833002B0EDB511E0320EE
:100A9000884280414042002807D1242B06DC0421F3
:100AA0008A1A0349CB18985C00E0002000BDC046BC
:100AB000E03B000010B5041C211C144800F0B2FA01
:100AC000211C134800F0AEFA211C124800F0AAFACB
:100AD000211C114800F0A6FA211C104800F0A2FACF
:100AE000211C0F4800F09EFA211C0E4800F09AFAD3
:100AF000211C0D4800F096FA211C0C4800F092FAD7
:100B00000B48211C00F08EFA10BDC0462040044066
:100B100024400440284004402C4004403840044015
:100B20003C400440404004404440044048400440AD
:100B30004C400440F8B51020FFF7BCFF094C271CBF
:100B4000143725786678281C311C002200F0F8F94B
:100B50000234281C311C012200F040FABC42F0D1C2
:100B6000F8BDC046083C0000F8B50B4C271C1437F4
:100B700025786678281C311C012200F0E1F9023446
:100B8000281C311C002200F029FABC42F0D10020C0
:100B9000FFF790FFF8BDC046083C0000F0B589B0F3
:100BA000002404900591FFF7C5FF022007210122D0
:100BB0000694079400F0C4F902200721221C00F0DB
:100BC0000DFA201C0B2100F0DFF9A04202D11823FE
:100BD000069301240021264D03916A782F78111C79
:100BE0000192381C012200F0ABF9381C0199002257
:100BF00000F0F4F903231F4E029314E0307871786B
:100C000000F0C2F9002807D103991B4AA3008A5CAF
:100C1000183369465A500134029A039B013A013352
:100C200002920393023EE30F00210122A2424B41B4
:100C3000DBB28B4202D0029B8B42DFDA381C019977
:100C4000002200F07DF90199381C012200F0C6F95C
:100C50000A4902358D42C0D1201E06D0069B049A57
:100C600005991360079B01200B6009B0F0BDC046D9
:100C7000083C0000DE3B0000E03B00001C3C0000A4
:100C800000B50A4B00211960094B01221A60196056
:100C90001A6019681142FCD0064B01221A60064BFB
:100CA0008022196852020A431A6000BD7080044015
:100CB00074800440788004408080044008B500F0CF
:100CC00031F90C4B03201A68120B12031A600A4BFD
:100CD0001A68120B12031A60084B1A68120B1203DF
:100CE0001A60074B1A68120B12031A60FFF7C8FF4D
:100CF00008BDC046008000500080015000800250B6
:100D00000080035070B5124A1249134800F008FEE3
:100D1000124C1348211C00F003FE201C00F000FEC2
:100D2000104E114D00242B196159DA68301C0B4B01
:100D3000143400F0F5FD642CF5D10C4800F0F0FD02
:100D400000F020FB011C0A4800F0EAFD70BDC0461F
:100D500018360000063600001C3C00008E3C0000E7
:100D6000303C0000493C000000000010543C0000F2
:100D70007B3C0000F0B53C4B8BB01D78002D3AD089
:100D80003A4B02901B6801209B685DE00134237898
:100D9000202BFBD0002B3AD0B30008336A469C507E
:100DA0000136FF2D01D135E001342378202B01D00D
:100DB000002BF9D1202B02D1002323700134012E06
:100DC0001BD12A4F2A4B06223B6001923D1C09E0B1
:100DD0002B680298196800F003FE002808D02B68E1
:100DE00014332B60019B013B0193002BF0D132E0C7
:100DF0003B681D7901E0041C2E1C2378002B06D0D3
:100E000000230722B2425B41DBB2002BBFD1002E90
:100E10001CD000E00025154C022E05D10398154981
:100E200000F0DEFD002801D0AE420AD82368124847
:100E3000D96800F075FD23681048196900F070FD4D
:100E400004E02368F0B29B6802A99847064B1B7820
:100E5000002B07D103E00198011CFFF753FF08485E
:100E600000F05EFD0BB0F0BD98020010A002001073
:100E700000000010883C00008A3C00006936000039
:100E8000913C000038B5041C154D0A2808D002D842
:100E900008281CD110E00D2802D07F2817D10BE0C4
:100EA0002B6800221A700F4800F03AFD0E4C201CEF
:100EB000FFF760FF2C6012E02A680B4B9A420ED9B4
:100EC0000A48211C00F02CFD2B68013B06E0074876
:100ED000211C00F025FD2B681C7001332B6038BDF0
:100EE0009C0200108E3C0000980100109D3C000008
:100EF00008B503E000F0B4FBFFF7C4FF00F0D2FB3D
:100F00000028F7D108BD000008B5034A034B044888
:100F10001A6000F005FD08BD980100109C02001049
:100F2000913C0000044B40211A680A431A60034BAD
:100F300001221A707047C04680800440A40200104D
:100F400070B50E4B061C1B780D1C141C002B01D118
:100F5000FFF7E8FF013E022E03D8094BB600F35815
:100F600000E0084B1A68012C03D1AC4014431C600C
:100F700003E00124AC40A2431A6070BDA40200103B
:100F8000083D00000080005038B50F4B051C1B7851
:100F90000C1C002B01D1FFF7C5FF0020032D11D839
:100FA000281C012302F02AFA02040608074A04E07A
:100FB000074A02E0074A00E0074A1068A3401840C9
:100FC000431E984138BDC046A4020010FC3F0050AB
:100FD000FC3F0150FC3F0250FC3F035070B50E4BEC
:100FE000061C1B780D1C141C002B01D1FFF79AFF67
:100FF000013E022E03D8094BB600F35800E0084B1F
:101000001A68012C03D1AC4014431C6003E0012496
:10101000AC40A2431A6070BDA4020010143D000051
:10102000FC3F005038B5084B041C1B780D1C002BEE
:1010300001D1FFF777FF23681822934323602368C9
:101040001D43256038BDC046A40200101F2342097D
:10105000184001238340181C014B9200D050704768
:1010600000E100E0054B3F221A60054B01221A60A7
:10107000044B40211A688A431A6070472480044058
:10108000D88004403882044008B5044B40211A68D7
:101090008A431A60FFF7E6FF08BDC0463882044065
:1010A00008B50320FFF7ECFD094B012252421A60FC
:1010B000084A1268002A00D01A60074B1A680132E9
:1010C0001A60064A00231360054A1360C04608BD33
:1010D000088204400C820440A802001004C00040B2
:1010E0003CC0004008B5FFF73FFD0A480021FFF76C
:1010F00099FF09480021FFF795FF08480021FFF7F5
:1011000091FF07480021FFF78DFF06480021FFF7F8
:1011100089FF08BD0840044000400440AC40044042
:10112000144004401C400440F7B50190FFF7DAFF7B
:10113000574B01991A68574B1A60002901D0564B3A
:1011400000E0564B564A04211360564B564C1A6821
:10115000564D0A431A60019A002A54D0544B002776
:10116000544E1F60544B301C1F60391CFFF75AFF50
:10117000381C09213A1CFFF7E3FE381C09213A1CF0
:10118000FFF72CFF4D4B8022196803201143196093
:10119000336807218B433360336802210B43019985
:1011A00033604B005B1899015B1801999B005B1839
:1011B00043490B60434B196801431960424B434953
:1011C000186801401960196809200A431A60FFF77E
:1011D0003DFF226880239B001A43226001213C4A84
:1011E000494211602A68324913432B60394B02226D
:1011F0001A60394B01221A601F601A601868104289
:10120000FCD001230B600720FFF720FF0820FFF729
:101210001DFF0A20FFF71AFF0C20FFF717FF0B2016
:10122000FFF714FF236880229343236022682B4B2F
:101230001340236022682A4B134023602268294B05
:10124000134023602268284B13402360019B002B2E
:1012500003D101221E4B52421A602B688022134395
:101260002B602A6880235B0013432B602A6880234D
:10127000DB0013432B602A6880235B0113432B6040
:101280002A6880231B0113432B6030BFF7BDC04683
:101290003882044034820440BF180000FF18000068
:1012A0003082044010ED00E00082044004820440DB
:1012B00004C0004064400440044001408080044079
:1012C00018C0004014C000403CC000400FF0FFFFB9
:1012D000088204407080044074800440FFFEFFFFD9
:1012E000FFFBFFFFFFEFFFFFFFF7FFFF08B5FFF773
:1012F0001BFF08BD00B5064B1A6801321A601B6857
:10130000013303D1034B1A6801321A6000BDC04695
:10131000B0020010AC02001000B5074B98420AD88A
:10132000064A00231360064A01381060054A13601C
:10133000054B07221A6000BDFFFFFF00B00200103E
:1013400014E000E018E000E010E000E000B50C4A16
:101350001368002800D10120C1438B4204D809E062
:1013600011688142FCD301E0591C081811689942A8
:10137000F6D203E01168C91A8142FBD300BDC04612
:10138000B002001010B5064BFA211868054B890011
:101390001C6802F047F8044B5C43201810BDC0469F
:1013A000B0020010AC02001037894100034B01224B
:1013B0001A60034B1A6801321A60704700C000407F
:1013C000B4020010034B01221A60034B1A68013269
:1013D0001A60704700000140B8020010034B012260
:1013E0001A60034B1A6801321A60704700400140CE
:1013F000BC020010034B01221A60034B1A68013231
:101400001A60704700800140C002001000B500283B
:1014100003D1044B01221A6003E0012801D1024BE1
:10142000186000BD044001400480014000B5002860
:1014300002D1044B186004E0012802D1024B0022C3
:101440001A6000BD044001400480014010B5041C36
:10145000002906D1164B96201968C00001F0E2FF62
:10146000011C002C0FD1134B8022186892000243FC
:101470001A60114B03221C60104B1960104B1A604C
:101480008022D20211E0012C11D10A4B802218686F
:10149000D20002431A600B4B00221A600A4B03224F
:1014A00019600A4B1A6080221203094B1A6010BDA2
:1014B0007880044080800440BC0200101840014045
:1014C00014400140C0020010188001401480014007
:1014D00000E100E008B5184B1A680E231340062BF4
:1014E0000DD1164B9E221B68DBB2134204D0144A66
:1014F0005360144B1B681EE0D9071CD501E0042B78
:1015000005D1104B1868C0B200F0BBF813E00C2BEB
:1015100006D10B4B8022596852000A435A600AE0F8
:10152000022B08D1054B1A68054B910601D5002204
:1015300000E001229A6008BD08800040148000404D
:10154000C40200100080004000487047C402001030
:1015500070B52B4C2B4B80229203DA67002190222E
:10156000061C201C00F009FA0023A36000F072F8AA
:10157000254B07251A68254CAA431A6019680122D1
:1015800011431960224B1968A94319601968114366
:101590001960204B802118684901014319601E4BD6
:1015A0001E481A608322226019681D4B1B6858432D
:1015B00001F038FF311C000901F034FF1949030A1A
:1015C000194A0B60C0B2032310602360174B1D60E3
:1015D000174B186860201C680440602CFBD101E0A8
:1015E000146800E001201C680442F9D1044B012278
:1015F0001A70104B802292031A6005230B6070BD95
:10160000C402001004E100E0A44004400C8000404B
:10161000A84004408080044098800440001BB7002C
:101620007880044004800040008000400880004032
:101630001480004000E100E000B5044A2023116856
:101640001942FCD0024B186000BDC0461480004017
:101650000080004008B5FFF777FF0023437308BD03
:1016600008B5FFF771FFC27B031C8218107CDA7B80
:101670007F2101320A40DA735A7B013AD2B25A739F
:1016800008BD10B5041CFFF75FFF837B7F22C318E2
:101690001C74837B013313408373437B0133DBB2C0
:1016A000437310BD08B5FFF74FFF407B431E9841C1
:1016B00008BD30B5002402E00570013401301D5D25
:1016C000002DF9D1121B131C02E00170013B013007
:1016D000002BFADCD043C0170240A01830BDF8B58B
:1016E000051C0F1C1E1C541E092B01D800240FE0E2
:1016F000181C0A2101F096FE221C031C391C281C10
:10170000FFF7EDFF041C2D1805E02F7001340135A3
:10171000013A002AF9DC301C0A2101F0C7FE303101
:101720002970601CF8BDF8B50C1CD9175F18061C91
:101730004F40551E092F12D9381C0A21002B03DAFD
:1017400001F070FE434202E001F06CFE031C211C1C
:101750002A1C301CFFF7E7FF041C351813E0002B90
:1017600000DA951E002201E0B4540132A91A0029C2
:10177000FADCEC43E4172C403519002B03DA2D2357
:101780002B7001340135381C0A2101F08FFE3031F5
:101790002970601CF8BD73B5069E041C1D1C300921
:1017A000531E00280AD000901A1C201C2B1CFFF787
:1017B000F2FF241805E0217001300134013A002ABB
:1017C000F9DC0F231E40092E01D8303604E0002D2D
:1017D00001D0373600E057362670013076BDF0B5BF
:1017E00085B0041C0F1C002801D0002101700025C9
:1017F0006BE0252903D021700132013405E05178D6
:10180000252904D121700232013401355DE03029EF
:1018100003D001320292202101E002320292029EA4
:101820009C4632782D3A50424241B6180296002228
:1018300005E00A235A438218303AD2B20136307892
:10184000031C303B092BF4D90296AE186346BE4206
:1018500001D97A1BD2B269280ED006D863282CD0C1
:10186000642809D058283ED119E075280AD0782874
:101870000FD0732837D11AE01E1D201C1B68FFF7FC
:1018800052FF04E01E1D201C1B68FFF728FF331CBD
:1018900017E01E1D1B68201C0093002304E01E1D82
:1018A0001B68201C00930123FFF775FFEFE71E1D47
:1018B000201C1B68FFF7FDFEE9E71A680120227073
:1018C0000433029A241801322D181178BD4201D236
:1018D00000298ED10023BD4201D2237005E0013CD6
:1018E0002370013D01E001256D4205B0281CF0BDCB
:1018F00010B50C1C131C6421221CFFF770FF10BDD7
:1019000000B5031C9BB00A1C01A8191CFFF7F0FFCF
:10191000632800DDFEE701A800F090F81BB000BDD1
:101920000FB407B504A901C90191FFF7E9FF03B09E
:1019300008BC04B0184770B50323041C184205D135
:101940000D1C041C194201D1934201D3002311E064
:10195000131C40CD043B40C4032BFAD8141FA40829
:101960000134A400032309191A400419EEE7CD5CE1
:10197000E55401339342FAD170BD30B50B040D0626
:101980001D430D430B021D430323041C93420DD240
:1019900018420BD1131C043B20C4032BFBD8141F8B
:1019A000A4080134A40003231A400419002301E011
:1019B000E15401339342FBD130BD00B5002300E078
:1019C0000133C25C002AFBD1181C00BD00B5031C0A
:1019D00001E0013101330A781A70002AF9D100BD03
:1019E00000B502E00130002B06D00A7803780131FF
:1019F0009342F7D0981A00E0181C00BD08B5FFF715
:101A00005DF90B48FFF788FCFFF78CFAFFF73CFB0A
:101A100096200002FFF79CFDFEF7F2FEFEF7DEFEC9
:101A2000044A0548111CFFF77BFFFFF76DFA08BD5C
:101A3000E02E00008E3C0000203D000010B5041C8C
:101A400002E00134FFF7F8FD20780028F9D110BD3D
:101A500000B50B4B984201DD0A4BC0180A4A8310AF
:101A6000D35C03220240082152008A1A93401A1CB8
:101A7000C0239B001A40054B1B5C101C184300BD83
:101A8000FF17000000F8FFFF4E3D00004E4300002E
:101A900008B54018511A013101F074FD08BD08B5B0
:101AA000801889189A1A0132FFF745FF08BD000017
:101AB00030B5B14B87B0D96EB04D4A1E91416A46E0
:101AC000D175A96A1A1CC806400F0138062807D824
:101AD00001F094FC040C1F1217191C00022409E0E9
:101AE0005A6E16329200D3581C1C15E05B6E1633EA
:101AF0009B00D45800230FE09B6DD46DA3420ADCF9
:101B00000AE0022403E00C24032305E00D24231C37
:101B100002E00D24EEE70D242C6148111F2800D9A6
:101B200022E16A461732944901F072FC200022003B
:101B300028002A002D002F003800400044004900F2
:101B400051005F0067006F00770085009300A200DE
:101B5000B400C300D500D300E300E600E900F100C3
:101B6000010105010F01110113011901081C00E019
:101B70008348191C221CFFF78BFFF5E08148F8E72A
:101B80000A1C0E3203E07E4809E00A1C1C32081CC5
:101B9000111C1A1C231C01F083F8E5E07948011C94
:101BA0000E391A1C231CFFF77AFFDDE07448011C74
:101BB0000E31EEE70A1C1C32081C111CF1E70A6EFC
:101BC0001020002A00D00A200A1C0E3206E00A6EFD
:101BD0001020002A00D00A200A1C1C3200946C46F7
:101BE000173402900194081C51E001201070086E17
:101BF0001022002844D00A2242E00A6E1020002A57
:101C000000D00A200A1C0E320EE001201070086E6F
:101C10001022002855D00A2253E00A6E1020002A14
:101C200000D00A200A1C1C3200946C461734029023
:101C30000194081C78E00A6E1021002A00D00A21C5
:101C4000504A68461730019002910094101C111CF4
:101C50001DE00A6E1020002A00D00A20494A009494
:101C60006C46111C173402901C390194101C0EE0B4
:101C7000096E012010701022002900D00A2241496B
:101C800068461730019002920094081C002201F06F
:101C900011F869E00A6E1020002A00D00A20394AA3
:101CA00000946C46111C173402901C390194101CCE
:101CB0003AE0096E012010701022002900D00A229B
:101CC000304968461730019002920094081C0022A7
:101CD0002AE0012010700A6E1021002A00D00A218B
:101CE000284A68461730019002910094101C002188
:101CF0001AE0009222481CE00092224819E00A6E85
:101D00001020002A00D00A200A1C1C3206E00A6EAD
:101D10001020002A00D00A200A1C0E3200946C46C3
:101D2000173402900194002000F0EDFF1CE00092B7
:101D3000081C002104E00D1C1C35081C0092291C05
:101D40001A1C231C01F03AF80EE0081C02E00C48B3
:101D500000E00C48191C221C01F049F804E0081CA2
:101D6000221C191C01F04EF86B46DA7D024B07B0BD
:101D70000120DA6630BDC04688040010241300102C
:101D800096040010A404001010B506490B1C8833FB
:101D90001A68141C1E34A4006050013203210A404A
:101DA0001A6010BD88040010054B0320191C8831EF
:101DB0000A68013A02400A601E329200D058704709
:101DC00088040010F8B5114D2C1C8C3420680130AB
:101DD000FFF73EFE0E4B0122D8629F6AAB6E061CD7
:101DE00002409A4210D1830703D420680230FFF7E3
:101DF000CBFFFF239B001E40B601BF10044B8C3568
:101E0000374301222F60DA600220F8BD88040010F9
:101E10002413001030B50C4B0C489A6A031C8C3309
:101E20001C68D3059B0E910500D5403B856E921032
:101E300001210A40AA4204D1E3188C300360024B0E
:101E4000D960012030BDC046241300108804001062
:101E500008B5084B5A1CD07F9A1CD27F0001120291
:101E60001043DA7F0333DB7F10431B031843FFF774
:101E70008BFF08BD8804001038B5FFF795FF0649B1
:101E800003230F22051C5C18154001332577001130
:101E9000072BF7D138BDC0468804001008B5FFF7FE
:101EA00083FF034B01228C331860024BDA6008BDBC
:101EB000880400102413001010B5064CA36E002BEC
:101EC00006D0FFF771FF044B8C3401222060DA60EA
:101ED00010BDC046880400102413001010B5064C35
:101EE000A36E002B06D1FFF75FFF044B8C34012259
:101EF0002060DA6010BDC046880400102413001072
:101F000008B5124B1B68002B00D09847104B5A693C
:101F1000002A15DD012A07D1DA69002A04D09A6166
:101F20000022DA610A225A615B690322191C91437B
:101F30000A1E02D0074A0121D166054A013B5361BE
:101F4000044B90331A68024B5A6208BD54030010C8
:101F5000241300108804001000B5064B5A69002AAB
:101F600007DD9A690F21044B1140D9771211013313
:101F7000DA7700BD2413001088040010044B597F49
:101F80009A7F090112020A43197F0A435A67704770
:101F90008804001030B50B1C093B012B0FD8084AF0
:101FA00000239C18257FC45CA54205D0054B083949
:101FB0005A681143596002E001330E2BF1D130BD54
:101FC000880400102413001000B508290DD0192929
:101FD00011D1427808231A4202D00022027002E096
:101FE0000F2303700723437005E000231A1CC2541B
:101FF00001330E2BFBD100BD10B50E4B596F0028DD
:1020000002D00F22914301430E244C4359679C3365
:10201000E418094B1B68292B02D0201CFFF7D4FFC2
:10202000044A0023E05C9918013308770E2BF9D19C
:1020300010BDC046880400102413001070B5124B68
:102040000F225C6F944304435C67104B1B68292B81
:1020500001D0082C17D00E2565430D4E211CAD195B
:10206000281CFFF797FF9C3E00239A19127FEA5421
:1020700001330E2BF9D1054B1B68292B03D0281CEB
:10208000211CFFF7A1FF70BD88040010241300106D
:102090002405001038B5104B104D1B68292B02D0B9
:1020A0006B6F082B17D0696F0E244C439C35641955
:1020B000201CFFF76FFF9C3D00235A19127FE2544A
:1020C00001330E2BF9D1044B1B68292B03D0696F08
:1020D000201CFFF779FF38BD24130010880400107E
:1020E00010B50D4C631CD87FA31CDB7F00011B02C5
:1020F0001843E37F1843E31CDB7F1B031843FFF700
:10210000A7FC0F23021C1A40227702111340001271
:102110006377A07710BDC04688040010044B5A6E48
:1021200016329200D258121A51424A41DA6670476A
:102130008804001000B5064B5A6E16329200D15832
:102140000139D150002901DA0D21D15000BDC0461E
:102150008804001000B5064B5A6E16329200D15812
:102160000131D1500E2901D10021D15000BDC0460E
:102170008804001000B5094B5A6E16329200D258EE
:102180000D2A03D11A1C2932127805E09A18507FC3
:10219000117F0001021C0A435A6500BD880400102B
:1021A00010B5084B0F245A6E16329200D1585A6D52
:1021B00058181440013104770D2902DC5B18121104
:1021C0001A7710BD8804001030B50F4B5A6E596D48
:1021D00016329200D2580D2A07D11C1C29342478BB
:1021E000F02008402043586507E09818447F057F99
:1021F00024012C435C650B114377034B9A180F2382
:102200001940117730BDC0468804001008B5044855
:102210000022011C1C390D23FFF741FC08BDC046FC
:10222000C004001008B504480022011C1C310D2315
:10223000FFF735FC08BDC046A404001008B50448EB
:102240000022011C1C310D2300F02AFD08BDC046F0
:10225000A404001008B504480022011C0E390D2307
:10226000FFF71DFC08BDC046B204001008B50448C5
:102270000022011C0E310D23FFF711FC08BDC046E2
:10228000A404001008B504480022011C0E310D23DF
:1022900000F006FD08BDC046A40400100C4A00234F
:1022A000111C46310B70111C47310B70111C483149
:1022B0000B70111C49310B70111C4A310B70111C31
:1022C0004B310B70111C4C314D320B701370704739
:1022D0008804001000B5074A011C042300208A1856
:1022E00004E0D1184631097840000843013BF8D298
:1022F00000BDC0468804001030B5074A0023891885
:10230000012206E0CC18051C46341540257040100B
:102310000133042BF6D130BD8804001038B50020FD
:10232000FFF7D8FF084C051C0021207FFFF7E4FFD2
:1023300025770420FFF7CEFF0421051C607FFFF7FF
:10234000DBFF657738BDC0468804001010B500205B
:10235000FFF7C0FF034C20770420FFF7BBFF607737
:1023600010BDC0468804001010B5054C0021207F28
:10237000FFF7C2FF607F0421FFF7BEFF10BDC0461C
:102380008804001010B5094C231C8C3318680130E8
:10239000FFF75EFB064B021CD8620F231A40227720
:1023A0000211134000126377A07710BD880400105B
:1023B0002413001010B5094C0021201C0D22FFF73A
:1023C00067FB201C0E3000210D22FFF761FB201C53
:1023D0001C3000210D22FFF75BFB10BD88040010AC
:1023E00010B50C4B00211A1C187F1C7801312043BA
:1023F000187701330E29F7D1936E002B08D0064BC6
:102400001B690D2B04D1137F111C29310B705373E1
:1024100010BDC046880400102413001010B50C4BEA
:1024200000211A1C1C7F18780131204018770133D5
:102430000E29F7D1936E002B08D0064B1B690D2B8C
:1024400004D1137F111C29310B70537310BDC0468A
:1024500088040010241300107FB500230C4A0D25BA
:102460001C1C1118097F01306E469955C60F854214
:10247000664176420133111C30400E2BF1D100230E
:102480006C46185DCA18013310770E2BF8D17FBD4A
:102490008804001010B5074B5A6E16329200D158BE
:1024A0005C1801392077D150002901DA0D21D15073
:1024B00010BDC04688040010034A0023111C94314B
:1024C00098320B601360704788040010034B0121A1
:1024D00094331A684A401A607047C0468804001056
:1024E000044A002313678C321360034B0122DA6025
:1024F0007047C046880400102413001008B59A4B9A
:102500000F20996A994A8B10184089110138525648
:102510000E2800D9C1E000F071FF08111A2327C06E
:102520002EC0C037C0C0C03B3F00002A00DAB4E074
:102530008F4B9A18403200239371A9E0002A00DAE9
:10254000ABE08B4B01209A1840329071A4E0002A36
:1025500000DAA2E0864B9A1840329279DA6697E068
:10256000081CFFF797FF93E0002A00DA95E0101CA3
:10257000FFF7D4FD8CE0002A00DA8EE07C4B596E28
:1025800016318900CA5083E0081CFFF757FD7FE031
:10259000081CFFF731FD7BE0002A00DA7DE0101C0B
:1025A000FFF75AFF74E0724B01209833186073E014
:1025B000FFF7E0FD6CE0FFF793FF69E0FFF726FE11
:1025C00066E0FFF7EDFD63E0694B00225A665FE0CD
:1025D000FFF728FE5CE0FFF7F7FD59E0644B0120B0
:1025E000586659E0FFF72AFE52E0FFF7CBFE0220C3
:1025F00052E0FFF72FFE4BE0FFF72AFC48E0FFF721
:1026000035FE45E0FFF7D6FE42E0FFF735FC3FE040
:10261000FFF738FE3CE0FFF79FFC39E0544B002207
:102620001A6635E0FFF7AAFC32E0514B012018662C
:1026300032E0FFF741FF2BE0FFF72CFD28E0FFF72A
:1026400045FF25E0FFF74CFD22E0FFF78DFE1FE080
:10265000FFF732FC1CE0FFF7C3FE19E0FFF776FE40
:1026600016E0FFF73BFC13E0FFF7D8FE10E0FFF7A2
:1026700015FE0DE0FFF744FC0AE0FFF75BFD07E005
:10268000FFF74CFE04E0FFF765FD01E0FFF706FCF5
:10269000012001E00120404208BD982BBED03EDC65
:1026A000382B9BD01DDC1C2B00D187E70CDC0C2BBE
:1026B00000D178E702DC002BEAD0EBE7162B00D143
:1026C00076E7182BE6D176E7282B00D17CE702DCF1
:1026D000262BDFD175E72C2B00D179E7362BD9D10A
:1026E00079E7662B00D18AE70CDC4C2B00D17CE724
:1026F00002DC3C2BCED175E7562B00D179E75C2B61
:10270000C8D179E76C2B00D17FE702DC682BC1D1FF
:1027100078E7762B00D17BE7882BBBD17BE7E62BD4
:1027200000D19BE726DCC82B00D188E70CDCA82B66
:1027300000D17AE702DC9C2BACD173E7B82B00D137
:1027400077E7BC2BA6D177E7D62B00D17DE703DC5A
:10275000CC2B00D09EE775E7D82B00D178E7DC2B97
:1027600000D097E777E7C046241300104E5B0000C7
:1027700088040010F32B00D17CE70EDCEC2B00D199
:1027800072E703DCE82B00D084E76AE7F12B00D185
:102790006DE7F22B00D07DE77AE7F62B00D16FE7EB
:1027A00003DCF52B00D075E767E7F72B00D16AE76C
:1027B000F82B00D06EE769E738B5184C231C8C3332
:1027C0001868FFF745F9211CE26E9031144B0D6833
:1027D000A2660022E2660135DA60032298620D608B
:1027E0001040251C1C1C022809D090420AD0012848
:1027F00002D0FFF783FE07E0FFF7E4FA04E0FFF7FB
:1028000057F901E0FFF706FB002806DDE368002B1F
:1028100003D18C352B681B182B6038BD8804001041
:1028200024130010034B0122DA660F229A775A779D
:102830001A7770478804001010B5054C0549201C14
:1028400000F0A0FEFFF7EEFF0123636610BDC04657
:10285000880400109C0E000000B5074B00201B6888
:102860000F2B08D1054B1A78824204D11868044B0B
:102870001840431E984100BD6400001088040010F9
:1028800000FFFF0038B5164B1A1C98321268002A58
:1028900004D0144B1D6801231D4001E094331D68D2
:1028A000114CA3689D4202D16268002A16D0002D07
:1028B00002D1002B0AD111E00C4B1B68002B02D077
:1028C0006168281C98470023636006E0074B1B687B
:1028D000002B02D0281C291C9847A56038BDC04693
:1028E0008804001070030010241300106803001007
:1028F00013B5002300930193244B1B68002B02D0D7
:10290000684601A998472249009B0878214A002877
:102910000CD0002B02D00223137035E01378013B5A
:10292000DBB21370002B2FD10B7009E0002B0CD100
:102930001378002B28D0013BDBB21370002B23D17E
:10294000154A1360154A13601EE014490968581AA5
:10295000444260414000107011484469021C002C40
:1029600004D08B4202D10A2343610DE000290BD130
:102970000A21516101999361D161084A1360064BA4
:1029800002221960034B1A7013BDC0465C0300108D
:10299000740300106003001058130010541300104B
:1029A0002413001008B5FFF7A3FF08BD10B5074CAE
:1029B00020600748016007490A60074A1360074B17
:1029C000029A1A60064A074B1A6010BD680300108D
:1029D0005C03001064030010580300106400001032
:1029E000A52900005403001008B5084B084A1968CF
:1029F00012688A1A1A6006D5FA2252001A60054B2C
:102A00001A6801321A60FFF73DFF08BD6800001028
:102A10005803001070030010F7B50E1C0E21051CA2
:102A2000019200F0AFFD1A4B03240C279E420FDDEC
:102A300009236B7301232B7328E0301C0A2100F05B
:102A400095FD301C29550A2100F03AFD0134061C81
:102A5000002E06D0E30F0022A7425341DBB293427F
:102A6000EBD1019AA31A033B2B70621B2B1C01E0D4
:102A7000195D5973013BD1180229F9D10F231C1B91
:102A8000002301E0013C2B55032CFBDCF7BDC046C5
:102A9000FFC99A3B38B50C4B01221A700B4B02222E
:102AA0001A700B4D0B4C08E01868884208D01B6860
:102AB0002360FFF799FFFFF71BFF2B682168024A8D
:102AC00010780028F0D138BD7403001060030010A6
:102AD000640300106C03001038B5334B334C1A1CE0
:102AE00094321268A061E161002A17D118280BD135
:102AF000C32909D12E4A12680F2A05D1181C383073
:102B00000E21162200F0B8F8A369182B04D1E3694E
:102B1000332B01D100F05AF8FFF784FE0A236361DA
:102B2000214C0123234D23678C34FFF745FE236896
:102B3000AB420BD003DC204A93421ED115E01F4A62
:102B400093420DD01E4A934217D104E0184B1B68E4
:102B50000B2B12D10DE0164B1B680C2B0DD108E08E
:102B6000134B1B680F2B08D103E0114B1B68102B74
:102B700003D1FFF787FEFDF7AAFA124B1A68124B32
:102B800010681968884205D012681A60FFF72CFF98
:102B9000FFF7AEFE044B1B6F002BC6D1FFF772FE92
:102BA000FFF778FF38BDC0468804001024130010DA
:102BB00064000010130D00006A0C0000790D000085
:102BC000990D0000640300106C03001070B5254CD3
:102BD00023681D68FFF75EFF23681A689542FCD0E2
:102BE0001E68FFF71FFE204B0A22204C5A61182254
:102BF0009A611522DA61231C903300221A60FFF7D4
:102C000011FE012323676436164C194D0AE0FFF7C5
:102C1000D3FD23682A681968914203D01B682B6092
:102C2000FFF7E2FE23681B689E42F0D10F4D18208B
:102C30002B1C90331C680021FFF74EFF0D4B6000EA
:102C40001968001900F03CFC3835011C0422281CCE
:102C5000FFF7E2FE044B18229A610022201CDA6181
:102C600070BDC046640300102413001088040010D7
:102C70006C03001058030010F0B501240DE0057836
:102C80000B1C254006E0C65CED0077083D43C554AB
:102C9000351C2540013BF6D5013A002AEFDCF0BD9A
:102CA00030B504E0845C8D5C85548C5401329A42CA
:102CB000F8DD30BDF7B5099D0AAC2678089F2C7861
:102CC00094461D1C002A0DD118E063465B5D4A5DE9
:102CD000D218131901920024B34201DB9B1B01247B
:102CE00043550135BD42F0DD0AE0CA5C12190024EB
:102CF000B24201DB921B0124C2540133BB42F4DD1A
:102D0000099B1C70F7BDF7B5099E0AAC2778089D92
:102D1000347800282FD000292AD01E1C9446002A7F
:102D20000ED1013F18E063469B5D8A5DD21A131BEA
:102D300000240192A34201DADB19012483550136F4
:102D4000AE42F0DD37E0CA5C121B0024561C01D1F4
:102D50003A1C0124C2540133AB42F4DD2BE0D15CB8
:102D600049420C1B211E01D0E1190124C154013339
:102D7000AB42F4DD1FE000291BD0181C002A06D14D
:102D80000EE00E5C135C0130F31A1C1BE40FA8422A
:102D9000F7DD10E0CA5C0133141B01346242544178
:102DA000AB42F7DD07E0D15C013349420C1B611EE9
:102DB0008C41AB42F7DD099A1470F7BD70B5049DE4
:102DC00001242C70141C002905D10BE0065D0A5D5E
:102DD00096420BD101349C42F8DD05E0815C00296C
:102DE00004D101329A42F9DD00232B7070BD00B589
:102DF00003E043185B78435401319142F9DB00232F
:102E0000435400BD00B504E08318013B1B78835494
:102E1000013A8A42F8DC0023835400BDF0B5114B1F
:102E20001A785B78825C1A4000D040220E4C0F4921
:102E3000231C261C04C32C3600221A6001240A1C01
:102E4000123117785578C75D3D4202D01F6827437D
:102E50001F60023264008A42F3D10433B342EBD1E3
:102E60000020F0BD61010010EC140010AD00001056
:102E700030B512234B43334A0131D3188A0051181D
:102E80001A785C78825C144204D02F4A5F2452186E
:102E9000947054709A78DC78825C144204D02A4A88
:102EA0007C245218533214701A795C79825C144273
:102EB00004D0254A7C245218A33214709A79DC7904
:102EC000825C144207D0204C5F226418251CA23576
:102ED000A1342A7022701A7A5C7A825C144204D07F
:102EE000194A7C245218A03214709A7ADC7A825CD7
:102EF000144204D0144A7C245218503214701A7BA5
:102F00005C7B825C144207D00F4C5F226418251C46
:102F1000523551342A7022709A7BDC7B825C1442D9
:102F200004D0094A2E245218A43214701A7C5B7CF7
:102F3000825C134204D0044B5918F43127230B70E0
:102F4000002030BDAD0000105C130010F8B52D4C12
:102F5000071C0025201C20214F22FEF70EFD002D0E
:102F600004D0221C7C23393223701370231C4F336E
:102F70000021013519705034052DEBD1214B2D2244
:102F8000181C38300270181C37300270A1209A705B
:102F90005A7040005F221A541B481A54A320400064
:102FA00019541A4908784978385C014204D0191C30
:102FB000533152330A701A700024211C381C01341A
:102FC000FFF756FF0A2CF8D1114D124E00242B7832
:102FD0006A78FB5C1A4201D0315905E03059FEF79E
:102FE000ECFC0D49091A0A310C48043400F0D4FAFB
:102FF0000235242CEBD10A49084800F0CDFA05200F
:10300000F8BDC0465C1300104101000061010010D2
:103010006C00001080000010630100109C14001070
:103020005E5B0000F0B585B001900027FDF7D6FB90
:103030006A4C3E1C6A4A7542754113687D19012B22
:1030400005D168480D210C22FDF788FC02E0002B19
:1030500000D1CDE0002303AA537023687F210B40E9
:103060005C2B00D198E02ADC382B00D18EE013DCF9
:10307000072B6AD006DC022B00D193E0062B00D090
:10308000B6E041E0212B00D184E0232B00D187E082
:103090001C2B00D0ACE081E04F2B4ED007DC3F2B47
:1030A00062D0402B62D0392B00D0A1E064E0542BD9
:1030B00076D05B2B3FD0502B00D099E06AE0732B89
:1030C00066D010DC662B3AD005DC5E2B56D0622B26
:1030D00000D08DE062E06F2B3BD0712B52D06D2B76
:1030E00000D085E02DE0792B4AD006DC762B4BD042
:1030F000772B3DD0742B7BD146E07D2B23D07F2BCB
:1031000025D07C2B74D135E031231370022E4BDD9A
:10311000231C083B1B681940542908D0032E43D0B8
:10312000231C0C3B1A687F231340542B3CD14C22A8
:1031300003AB1A7038E0322335E0332333E0342315
:1031400031E035232FE036232DE037232BE03823E1
:1031500029E039231370062E26DD231F1B68194032
:103160004723232920D11EE030231CE02D231AE021
:10317000412318E0422316E0432314E0442312E0E5
:10318000452310E046230EE048230CE04C230AE0E0
:10319000502308E0522306E04F2304E0552302E0C9
:1031A0004E2300E049231370ADB203A8291C00226E
:1031B000FDF748FC23681A0605D5E91D89B20A48BF
:1031C0000022FDF73FFC2368DA0572D50735A9B266
:1031D00006480022FDF736FC6BE0C046EC140010F8
:1031E00070010010DD370000C93C0000665B000084
:1031F00023680122134206D0A818C0B2002107227A
:103200000223FDF78BFB23680222134205D0A81D81
:10321000C0B200210623FDF781FB236804210B4285
:1032200005D0A81DC0B202220623FDF777FB236854
:1032300008210B4205D0681CC0B207220223FDF70B
:103240006DFB2368DA0606D5681CC0B20421022291
:103250000623FDF763FB23689A0606D5681CC0B2F7
:10326000002102220623FDF759FB23685A0606D5E2
:10327000681CC0B2042107220223FDF74FFB23681C
:103280001A0607D5281C09300222C0B20821131CD7
:10329000FDF744FB2368DA050BD5EDB2281C093095
:1032A000C0B20B210A35FDF723FBE8B20A21FDF776
:1032B0001FFB013604340C370B2E00D0BAE61B4836
:1032C00003210622FDF74AFB194D1A4E1A4F00241E
:1032D000019A2B78D35C6A781A4205D0A3009859DA
:1032E000395D0922FDF7AEFB01340235092CEFD11F
:1032F000FFF7B2FA002814D006240321201C00F0A6
:10330000DFF80321C5B2201C00F030F9281CC9B237
:10331000FDF7EEFA092C01D10B24EEE701340E2C57
:10332000EBDDFDF765FA05B0F0BDC046983600004C
:103330006C00001074010010A400001070B5041C93
:10334000FFF76CFD201CFFF76DFE0A4B1B78002B6E
:103350000ED0201CFFF7FAFD074CC8235B00074E78
:10336000E518211C301C5034FEF7DAFAAC42F8D1D3
:10337000002070BD750300105C130010693600005A
:1033800008B5002805D0FDF708FA0748FFF7D6FF73
:1033900008E0FDF70AFA054B1B78002B02D0044821
:1033A000FEF7BEFA08BDC046A20500107503001066
:1033B000685B000000B5FEE700B5FEE708B50A4B04
:1033C0000A4A0B4903E010780132187001338B422E
:1033D000F9D3084B0849002201E01A7001338B42EF
:1033E000FBD3FCF77BFFFEE700000010BF5B000093
:1033F00098010010980100101815001002B47146D1
:1034000049084900095C49008E4402BC7047C04627
:1034100003B47146490840004900095A49008E44E6
:1034200003BC7047002934D00123002210B4884225
:103430002CD301242407A14204D2814202D20901E3
:103440001B01F8E7E400A14204D2814202D2490004
:103450005B00F8E7884201D3401A1A434C08A042A7
:1034600002D3001B5C0822438C08A04202D3001B3D
:103470009C082243CC08A04202D3001BDC08224354
:10348000002803D01B0901D00909E3E7101C10BC78
:103490007047002801D00020C04307B4024802A1B1
:1034A0004018029003BDC046D90000000029F0D0AA
:1034B00003B5FFF7B9FF0EBC4243891A1847C0464F
:1034C000002941D010B4041C4C40A4460123002222
:1034D000002900D54942002800D5404288422CD31B
:1034E00001242407A14204D2814202D209011B0116
:1034F000F8E7E400A14204D2814202D249005B0015
:10350000F8E7884201D3401A1A434C08A04202D37C
:10351000001B5C0822438C08A04202D3001B9C08BD
:103520002243CC08A04202D3001BDC08224300281F
:1035300003D01B0901D00909E3E7101C6446002CE5
:1035400000D5404210BC7047002806D003DB0020A5
:10355000C043400801E08020000607B4024802A1F1
:103560004018029003BDC046190000000029EBD0AE
:1035700003B5FFF7A7FF0EBC4243891A1847C046A0
:103580007047C04600B5002905D0002301390370FB
:1035900001300029FAD100BDF8B5041CA30719D1E8
:1035A000231C04CB0F4D104E50199043021C201CBD
:1035B00032420FD1181C0B4F04CBD519954335421D
:1035C00008D1181C074F04CBD51995433542F1D0CB
:1035D00000E001300378002BFBD1FEF7F7F9201C47
:1035E000F8BDC046FFFEFEFE8080808053455249F4
:1035F000414C20434F4E534F4C450025732072657C
:103600006164790D0A00444D31314343000D0A4293
:1036100079652E2E2E0D0A0056414E494C4C410024
:103620007631002578000D0A253032782020000DF3
:103630000A413A2000202025633A20000D0A4D3A25
:1036400020002020473A20253032780D0A005761AB
:103650006974696E6720666F7220646174612E2ED2
:103660002E0D0A00526561642025730D0A004F4B30
:10367000004641494C454400656E61626C656400DA
:1036800064697361626C6564004C434420646562E4
:1036900075672025730D0A00030300000003030073
:1036A0005C0003030C000C03037C287C03037C44B4
:1036B0007C030324104803032854080303000C0070
:1036C00003033844000303443800030320100803B5
:1036D000031038100303804000030310101003038D
:1036E000004000030320100803033844380303009C
:1036F0007C000303645448030344542803031C1050
:103700007C03034C54240303385420030304740C37
:10371000030328542803030854380303005000030C
:1037200003805000030310284403032828280303C0
:1037300044281003030454080303384C5C03037843
:10374000147803037C5428030338444403037C4463
:103750003803037C544403037C14040303384434C7
:1037600003037C107C0303007C00030320403C0324
:10377000037C106C03037C404003037C087C030340
:103780007C047C03037C447C03037C14080303381F
:10379000447803037C146803034854240303047C23
:1037A0000403037C407C03033C403C03037C207CFB
:1037B00003036C106C03031C601C030364544C0370
:1037C000037C440003030810200303447C0003032C
:1037D000080408030380808003030408000007082E
:1037E0000400000000BF01BF010905000007000739
:1037F00000070007130A00002000E400FC003F005F
:10380000E700FC003F002700040F0800000C011E29
:1038100001FF03FF032201E201C2190D00000E00A7
:103820001F0011019101FF007E00FC00FE01130149
:103830001101F001E0140A0000EE00FF0111011176
:1038400001BF01EE00E00130011001050300000F8F
:10385000000F0A050000F800FE03070701040B062D
:103860000000000001040707FE03F80F0800000035
:10387000000A000E001F001F000E000A11090000C0
:10388000100010001000FE00FE00100010001008D4
:103890000400000004800780030D070000100010E2
:1038A000001000100010001008040000000080014B
:1038B00080010D07000C000FC003F0003C000F005A
:1038C000030F080000FE00FF01010101010101FFDB
:1038D00001FE10080000000002010201FF01FF01CB
:1038E00000010001100800008601C70161012101EB
:1038F00031011F010E010F08000082008301110138
:1039000011011101FF01EE11090000300038002CF7
:10391000002600FF01FF012000200F0800008000AA
:103920009F011F0111011101F101E10F080000FCCD
:1039300000FE010B0109010901F901F00F08000067
:1039400001000100C101F1013D000F00030F08005B
:1039500000EE00FF01110111011101FF01EE0F083E
:1039600000001E003F0121012101A101FF007E088E
:1039700004000000008C018C010804000000048C8D
:10398000078C0312090000200070005000D8008846
:10399000008C01040104011109000048004800489E
:1039A0000048004800480048004811090000040190
:1039B00004018C018800D80050007000200D070021
:1039C0000002000300B101B9010F0006190D00004B
:1039D000F800FC010603FB06FD0505050505FD05D0
:1039E000FF050601FC01F8120900008001F0017CCE
:1039F000004F004F007C00F00180010F080000FF25
:103A000001FF01110111011F01FE01E01109000078
:103A10007C00FE008301010101010101830182118B
:103A2000090000FF01FF010101010101018301FE05
:103A3000007C10080000FF01FF01110111011101BC
:103A4000110111010F080000FF01FF011100110019
:103A50001100110001120900007C00FE0083010129
:103A60000121012101E301E20112090000FF01FF30
:103A7000011000100010001000FF01FF010A0500F6
:103A8000000101FF01FF0101010B0600010001011E
:103A9000010101FF01FF10080000FF01FF013800D4
:103AA0006C00C6008301010110080000FF01FF0146
:103AB00000010001000100010001160B0000FF01E0
:103AC000FF010F003C00F000F0003C000F00FF0180
:103AD000FF0112090000FF01FF010F001C00700030
:103AE000E001FF01FF01130A00007C00FE008301DA
:103AF0000101010101018301FE007C0F080000FFAC
:103B000001FF012100210021003F001E140A0000D6
:103B10007C00FE0083010101010101038307FE0413
:103B20007C0412090000FF01FF0121002100710047
:103B3000DF008E010001110900008E009F011101BC
:103B4000110111011101F301E2110900000100014D
:103B5000000100FF01FF0101000100011109000047
:103B60007F00FF008001000100018001FF007F1144
:103B700009000007001F007800E001E00178001F45
:103B80000007190D00000F007F00F001E0017C002C
:103B90001F001F007C00E001F0017F000F120900F0
:103BA000008301C7016C00380038006C00C7018336
:103BB0000111090000010007001E00F801F8011EB4
:103BC00000070001120900008101C10161013101FA
:103BD00019010D010701030100070008000A010097
:103BE000181110133831303378717073C8C1C0C3E5
:103BF0008881808384848782C5C4C7C275747772C4
:103C00003534373215141712020702080201000377
:103C10000109030402040205030500064669726DEA
:103C2000776172652025735F25735F76310D0A0019
:103C3000436F6D6D616E6420202020446573637254
:103C4000697074696F6E257300252D3130732025DE
:103C5000732573000D0A5479706520273C636F6DDE
:103C60006D616E642D6E616D653E203F2720666F2D
:103C70007220706172616D730D0A00557074696D08
:103C800065202575730D0A003F0025730D0A0D0A86
:103C900000564F5941474552203E3E2000256300C3
:103CA00048656C70004E6F20706172616D73004BDF
:103CB0006579207072657373003C6B6579313E20C5
:103CC0003C6B6579323E202E2E2E0044756D70209F
:103CD0006D656D6F7279006C004C6F6164206D656D
:103CE0006D6F7279007400546F67676C652064694A
:103CF00073706C6179206F757470757420746F20A7
:103D0000636F6E736F6C650000800150008002501D
:103D100000800350FC3F0150FC3F0250FC3F035029
:103D200025735479706520273F2720666F722061C4
:103D3000206C697374206F6620617661696C6162C2
:103D40006C6520636F6D6D616E6473257300A132C5
:103D5000C205557520C5F00E3EEB55010EDC322B29
:103D6000101713439CC7042B010456116A195649B6
:103D70000A20C06A11C883C80C4EB939B70C560561
:103D8000AED3CD364051501711899D5062CC5502AB
:103D90001B555532D0941D4D557307254D1A6F9EF6
:103DA0000978490C4CFB80C030713C555D052120E1
:103DB00053232E85101EEC1C1025440BB03C8300B1
:103DC000E41101C664A401422440C40B50559580FF
:103DD00014510154048E269A3222A29D888C62AC22
:103DE0000771C45550C40210820881303363341CFB
:103DF0000E4EB3A4200331318D8D0C4C50C700887A
:103E00000A7FE23B5474774C996E5F2F0CDF5304AA
:103E100048280A810C65B90F00000000000000006E
:103E20000000208000C06CC3C810020000C800223F
:103E3000218C84080B818840884097601F13B361F0
:103E4000FB700BECC0320F7FBC0F51140511458481
:103E500084B8BBAAABBB008022303323227389BB5A
:103E600084B4BB999999457754B5B7555555DB2519
:103E700090DC3E333221404040CE9808029244000C
:103E80002000CC8012E034139200361583AFFC1072
:103E90001C303028DE4438647D1374C637408840B7
:103EA0003EF603122204045000FB0CC88CCC4021C7
:103EB000C03AA1A7201364754E59647D7F72D8C99A
:103EC00032E24A3B0088030100745C28E2548D749E
:103ED0003B143C1141324074F3E23E1283D2C9409C
:103EE00009CC44C25C0E08D8FDDD335D7C13163965
:103EF00063CA6704110002212211510222C1408CC1
:103F000084423B6BFC34FD642881F5A585001E8C42
:103F1000CECFCC221C23A0C4C8A2AC20FC4CCCAE7B
:103F2000CB328B0CCE374F44C8C523FF8E3FE13CCC
:103F300023C1E8B4E0BC23F01F4F214828D6D8E0C5
:103F4000C8C808CBBA40424C80EC8B0C8DC03242C2
:103F50008AC800C32C33CA5020874014121E7371C4
:103F600017611CD5015B853FF40D3E45394B01833C
:103F700033013E1308A54C2228358F1F02F0D8D8F4
:103F800027CB28C388030B13F5333C2C2F0EC520F9
:103F9000484D43C1791483C58244D390800389334B
:103FA000958040D4400022DEA7330408021B964FC0
:103FB000C5E04C1582113510BBD34C1965845325CF
:103FC0005D5D56544D14404053544B00C1C40184B0
:103FD0008C20CFC401C48C155F244C8A30CFC4F42C
:103FE0000068233C08E0D91D540140E2C861141167
:103FF0001340D113D30DC8014C723C2FCEA7E485DA
:10400000DAA94F92F030B230A2333332C333C30255
:10401000CC0BD80CA04C124F1555080814E8C8DB7F
:10402000EB7A8721B4CCF4804A0DEAB5F2D43DC4D2
:104030001352FF04205998936EFAE240DA8A49300D
:10404000380CC3F0183322238C1A245F5515000056
:10405000032300120311710008843C03CC480800BC
:104060007783DA00301300002C202101306088ECC7
:104070000C041011812448C24B8C0002C43009800A
:10408000C404F0C83832322021808ABB32322A443C
:10409000B8E2A00E82326121FB402633618D2048B8
:1040A00053D1208C1510234228C41812FA00082579
:1040B00000019248408000C784041402020404886E
:1040C00003100002082000824888400C09012108E2
:1040D0000058E5C110FFD27520D11372700E809484
:1040E000A2FC3D3048C0D280C4F4832C82A832B1F7
:1040F000110641F4A1636C72890C2123491000A1BF
:10410000109022F9E41F25CD03178282C3CCEF0360
:10411000C440200081A518306D83DD3BCD5060C4C4
:10412000A02830C03CE05042853D0F3676FFCF33AB
:10413000ECCCCC08030310CC001EDAF1B0032CC287
:10414000F212832CCB31C034C36058F9BE26C38829
:104150008F2309400808314800C920580515FDC4BF
:10416000BF20157F505401C41853FC90186081453E
:10417000BD430B02110208082108084C10030E0869
:10418000017D3E1636F1344144639311D3B443A408
:10419000328004AE38BF47B807FF378E8B2C71C70B
:1041A000D9B80F1423EF43324BC37B1344AC8F8237
:1041B0008BE201C82FF4D47E00601340300E7814D7
:1041C000416FB7208AC7389B840420213676B133EB
:1041D0000080618B843B44817B7550B2C46D02507A
:1041E00008800C03648816638295D5444221350308
:1041F000A4041D6014072029D0D90A80120312EEEE
:104200002F548AC2009084A60C50AC928401A7D48B
:10421000C8317E8058903DC81074ADBB57CA33FC7E
:104220009CD68488331D4104220FF312321193125D
:104230000F648ECF14C084840371C8717CCF0B339C
:10424000D77333B8CA7AEB0633C40FAA9501228418
:1042500003CB443230A38BC2A24F8C80000EB0350A
:104260009380408E4C001601C18D6098408E088668
:104270002806D0444C047A2023223010082321C77A
:1042800084C48EA1C4EC311DF1004C52C20087C021
:10429000078000F18F17C048902C04D5403220D5FC
:1042A0004020720C40C354040133F94B3338E2CC44
:1042B000382D55F68010428D33F600829404F0CEEE
:1042C0000908450432B68C8CA58C2455C80856C8FC
:1042D0004852C8085600252341953222563282544E
:1042E00029236B1532A204C45010054451151155F1
:1042F00049C5A878491055111551505654155155B6
:10430000D151455785542E101714270403008008F7
:104310008040E0E7921BFFFF375D8C2903C8B7742C
:10432000C2503C8109A036A0C2C8002108F479120D
:104330008273778B4058AED462A03E9040C18374A4
:104340004408019190018F730C49558F3F03CF4E64
:104350007038EEFF710CC50C6E0484A50200CAD43F
:10436000017E0304C002244E203C063018E06500A4
:104370006660E0C54E1CE020DB4E5C2650E0A2DA11
:10438000357D13F800DB6B710C6500668784C50C06
:10439000910C0404448465003075666330176673BD
:1043A000301266B15E3014665B2666B788910CC524
:1043B0005C8CEF1348F073146381004B60001CC3E6
:1043C000367C14EDABDC72DC101EF81EE8BB31B598
:1043D000E47AF3E90EE960BD4CF0E8AE1144F0D4A4
:1043E0001B0404448404446E6D2C6E0CEF048C0199
:1043F0002329080D085C06A14E4E20305ABC70E0FF
:10440000E0DC50D4F34CA0EEE00D084D320023DF89
:104410003C7B1E1F00DD3F9C10069C025C8CFF9CB9
:10442000A2E61C10762127A9266666D4A3FD089C67
:104430003002667743A6E6A6F9083BCC4F14F71482
:10444000E7541BCCE766CC3F14B10714135C6666D7
:104450006666CC3FD42F14F7E1086666666666662A
:104460006666CC47563794235C514E6666CC9F54A3
:10447000BF540B562B3010C6BB66E63B1C629CC378
:10448000065CB366CC2754250366CC93FD089C429A
:104490005B5C83560FD43F945F945BA09CA2A260A8
:1044A000739C2B5C444C47E616B6DCD4EB86A644E2
:1044B00054F12BB122E64816A14E30A69B30059C44
:1044C000022746466646463B66666666D4AF14B724
:1044D00054A70C5FCC5BE616767686485C43CCBB73
:1044E0005C131CE508C43106FD089CD3FD08C8DB3D
:1044F000CCBFD4CFFD08C823FD0866665C7D06FDF1
:10450000081CDBCC312FD43F8C4D1F5441535C0130
:104510000ACC3D1FD43D0BCBCC37F846E8D4311F35
:10452000E91ECC77D4F92B53CC3FD41F63CC0FD4E6
:10453000E7F3CCD7D477BBA6CCE7D4E77B30A7850D
:104540000614DFCCC7D42F23666666666666666689
:1045500066CC2FD41F5C131CE50865066666E1086F
:10456000DC49066666E1089C3D06CC9FD4EF94BF0B
:10457000D3D4BF9487D45D0714E714D7CCEF5BD4B2
:10458000479407143F14CF546FCCAFE906CCB7D48F
:10459000AFFD081CA3C49CA27D07305F5C8506307C
:1045A0003FDB66666666CC13668106309F7BCC195E
:1045B0002FD4652FFD081C4506CC27C8D43B9C1B77
:1045C000DCC444C4A14E5C44E616864BDCE90876A4
:1045D000E044844484C4C4E0B0EE8C6084049C98BD
:1045E0001CE2330862E21388A0069CA2CE660CEFA0
:1045F00056AF301006B326061F6606E908F613DC30
:10460000050C1E56D7EB668666468F0866E90805D8
:104610000C8CA7F623A08676A69CEAEAEA43FE1F46
:10462000FA538E26F3FBE676A63030C6FB46C6C6A6
:10463000FB46C65C13A2A6E77EA066D46062BBBB45
:104640007EA646EF600684E0B05E5CD4A6F3E00E82
:104650000A5A137E0ABEBAFE930CBB26F64B76F6B8
:104660002FB00E1E5B36A6CEA6061E1A60AA06A0A6
:10467000E026D49B133373C38382C272321210308C
:1046800070C08087C7773717113171C18184C474B6
:104690003414183878C88884C57535158D40A86BD2
:1046A000D14C53AE4E70382B8D405D40AEE04E5C29
:1046B0006650293A8CA0BEBEBEE0C9402D409D4C3C
:1046C0004140C9400E882BC940B0AED14C2138784A
:1046D000B5407140F938A140D14CF82938DD40355A
:1046E000409D4C8D4C8C60BD4CAE28C9404540F976
:1046F000387D4CD1402D409D4C11445D4038E03018
:1047000051A6A64E70F866A030049C58300B991C38
:10471000C4C4A0706E1C5090D0814E0E5C62E076D6
:104720005A5CD0D0FC30F65A56E060A09D0CCC60AC
:104730006000C8CCF73004C8CC66EBE00000BC8851
:10474000E4E8D8787CA8FCF844404CF474000B31C1
:10475000B132A434D732BC168D34C43689238824B0
:104760008A25A711AD123B13C41443159326FA31C1
:104770009633C934CC3543168026CF368223832422
:1047800084255411AB12AF13A91405158F26BF0051
:104790009001AC02A203992392337F36EC07EE0816
:1047A000F10979406A30642071107E49D6487C0056
:1047B0008F01AB0297039E041B051A06DF44E044F9
:1047C000EA16764067306D205E10FE49FA48CA0A44
:1047D0000ACAEAEA4A8C330E060E46E04ACAEAEFF3
:1047E000E00050404E30C12012107F491248019322
:1047F0006693029432940095459503498136B0FA48
:1048000013FE2388C85E9D38D140C14C0ED5405D53
:104810003C690CAEB05E593CFAEF0EDBCC1FC8E031
:10482000C4E08D40AE88FE13485E5D40FAA00EE302
:104830003910E32E0E7AFE4B48CC33CC23C4884487
:104840005CA606E641174687CECE235C62EE4F4C4F
:10485000078D180EA6AEAB4C653F213C39106ECECD
:104860005C5A5E26E6433ED454D3EEC116D84E3E83
:10487000CE6BAED8221ED8AEAEBEEB1E2EAE8ECE06
:1048800093D83ED86EEED454B3EEB13C6ED8469C6D
:10489000EE6514EE132E62F38E42FA03DC9B4CCBD2
:1048A000D140F540A140FD40F9381E5D3CB05E5856
:1048B00046353CA606E631164116DC6654EB5E9D95
:1048C00038CC3BBEBE711829408C2B711829404C46
:1048D000776666009D3C8C3F4E5C665029384C13D1
:1048E000BECC604484991A4E6E5E546F94E7D41F18
:1048F0005447145F9CD09CE0DC9090109050901036
:104900005030165CE09094F36B1CDD149C505C10EE
:104910009CE05CDD149C50DCE05CDD145CE01CDDA4
:10492000141CE0C8488D40AE0E2EBAFE43884C1BC6
:10493000CC13485EEE4CC91B8C2BAE0ECECE4E5C1B
:104940001050EE66F62F661B268EEE58EEEEEECE7B
:10495000EEF69F8EFB2EEE66DB4EEE98EE4C1B8E37
:10496000CEEE8E5B2EEE98EE4C0BE6F7EEEBCC47E0
:10497000C84C1F48734463C44CC38C1B842B881BD6
:104980008D184B6E8E0039103B26F6278EB32E669F
:10499000009D384C5F98EE6600613C71183138D844
:1049A000AE0E263B6EEE3BD454B726E36E4EEE655C
:1049B00014EE133E8EF32ED4CEEE549BD88E8E4E34
:1049C0005C50D89C90905B8A8ABEEB1ED8AE4E2E6F
:1049D000D88E1E62ABAEFAAEFA237E661E8E9B9810
:1049E000CC67CC53213C3BB05846353C5D40ED385C
:1049F000CC1B690C11448C1BBE00690C0B5ED8AE3D
:104A000098AECC1FCC1F866EDAC3D8993C4C7BD1B4
:104A100040E1403138F5405D3CCC6F213C4CA0BEBC
:104A2000E04E5C7A360E8E4CA0234ED88D18EECE1A
:104A3000E05C4ED01050D050105090D0D050D0509C
:104A40005CE0F8448460FEFE2BFE174888B0A0E0CE
:104A500030E5A6255060E6B356069F4D4E2D2C8CB2
:104A600063B8E64B66A646A830FDA91C8932EE4E17
:104A700070DCD010901010D01010684E5C1010D068
:104A800010D01090A8EE30E00835508C337D2CA962
:104A90005CBBE6E784EEBBE94CB30D08355008E695
:104AA00053F12C8C1F8884A95C8BB806F8A6E8A368
:104AB000EEED2C7D2C065670389C1A1EA6EEEE6E7E
:104AC000762BDCDCEEEE76DB5636DCAAAA6E2AAE5E
:104AD000F025501C6A27352C7B869C0AAE7CEE663E
:104AE000AB2550D8F8E60122761C1BDCDC76EB56B1
:104AF00070EE38AEEAEA8E8ED86E1C6A93AAD8AEF3
:104B000070AE383CAE9C6A2670AEF0A6986BAE7064
:104B1000B6567F4EF02550F12C3550F12C352C59DE
:104B200002EE930C1720608C604C1F5D4004881AC5
:104B30001EBA4EE0A630DFA656602E1C6A6AA07030
:104B4000EEF0EECB314498D44AFA1BE6FEE00D08B5
:104B50003550512C1EBED05CA2E663212C8C23E183
:104B6000202B88E12084068C95030D54910CE021C4
:104B70002C0C811C0ED8AE8C75038C891F0D08A6D9
:104B80004E3089BC70A66056064E701C30FA621F0B
:104B9000061730A80637624330B0C6161C10AA8C20
:104BA000812B58EABC3006461C101006BC709806D3
:104BB000B0A0E0E68C7D3A5CD0D06B621F02D3E6F9
:104BC0001C4662A21B88A29076678C55021C10902E
:104BD00090505CA12636763F8C835C90905336765D
:104BE000E1238C3B5CD090492AC88C7BA0DD4CD95A
:104BF0001C0EFEB7E6734EDC905050A646171A9571
:104C00002A60EEEE5EAEFCAE9B88465E7C464BFCB8
:104C1000A6462BFCA6464F06F12A86095435508439
:104C200044CCC92B6E0C470C3708412C0922B8FE26
:104C3000239C514E7D2C0E76B8EEEEBEEE66AEE8AD
:104C4000B8A6AEA875021C02FD263676DFA202E2E7
:104C5000578C239C10EBA61C5013024213A28C23EA
:104C60009C101B8928702B367647A202E2878C4B5A
:104C70009C501C1090D0552AA61C90DD2602421391
:104C8000A28C2B9C5021268928A6B0A2AE3CE855C8
:104C9000023676FF8C635C105065222940DD4C8B18
:104CA000488C3B6262B7B9281B0D282940EE70384A
:104CB00039023676478C53BEF336769F8C2B9CD0C8
:104CC0009126A61C105859028928B03CC536A0620E
:104CD00062608CAB9C901C10D0D0A1263676CF8C15
:104CE000635C10102D26DD4CB0F089268C3B62628F
:104CF000B7B9281B0D289B3676078C1BBE23486B43
:104D0000B616F6E7F623A2F6BF1926A28B901CB6BC
:104D100016F6F6F6F62F8CA7C2A28C2FC23000B67C
:104D2000D6D6A7D62FD6DF8C235C50138C23B92878
:104D30001B0D28593C238C535C10101C10105C5523
:104D40002A8C23B928930D287B8C235CD06B8C2371
:104D5000B9281B0D28BE0019401144D485321C51BE
:104D60004E8C235C90438C23B9281B0D282138538B
:104D70004E70F8BC62AEE07A6730FD63DD4C5ED900
:104D80001C1A66F657E6F74E5C901A6348FAAEBCFA
:104D9000A68646581C90A2A6464C13906046255005
:104DA000E62B56064D4EA670EE38AEB0A0E0EA26D1
:104DB000BC30061C426BA2BC1C10B61B9013D090DA
:104DC00090C3FC5A7A7C5CE227D05C139CB67F10BF
:104DD000B64FB64F3066663B50239013D00310F3A6
:104DE0001CD0D01630A006CFC6E676541B5C23FC40
:104DF0009CD08C1F501390EAAA1C224BD01CAAE016
:104E0000E65CD0A362A6DC50BEA3468384A04E30ED
:104E100004060B3007603AA0C6E346603A3A9C426B
:104E20001F467A1ABA5A463CEEEEB6A62550E6233D
:104E30001C4A235C514EEA273656CB8C3D23355015
:104E40000C3F0C2FB85EA84EA6E881328C27880153
:104E5000228459020C1F08DB04CB8C9503B05E7EC4
:104E60000E0D54910C45364E7E7EEE25500EE69B7F
:104E700030F41C0A7362A22F30EBCA2B4AAAEE3E12
:104E8000EEFBAE512C0A4E9C90D0AEA05ACE1C50D8
:104E9000FE5C50D01CD0D090D0D0602B9C509C4257
:104EA0004E1CD0B656FCA6BC430C1F0CAB255006BE
:104EB000F8661F4663601CE65316D0164BB636DC08
:104EC000F0E030FCDB661C50BB25500E30F0E6668F
:104ED000952AAE9D2CE0355006567038B6B660CE99
:104EE000CEE3AED8AE5E5A0EE6EB9C5062D0BAA0CE
:104EF0005A76F3DCD060269CA0DA6062E31C223F85
:104F0000A05C5050905A605CAAE076F65F1CD02AF4
:104F1000A630FDA66A1746F0E026233550E6255058
:104F20005EA84EE6E8E0B0BE0E4E5CD01940FE1B17
:104F3000FD40D91CFE134EE04EBE2626D84EDC5056
:104F400050905CE016CAA78D4FB7A6D0A14CC848B8
:104F500001504C378C33350CBB8C605EAD44D14076
:104F60004CA3B14CF5402940CC47810C0EB01EAE8D
:104F7000E0A140D140213CE940CC1F810EB14C6BF7
:104F8000350C1140D140B0350C1940ED385D3CE98D
:104F900040694E01508C600E5CA24A2F4E7A366BEF
:104FA0000E19401ED140B05E350C1540E140693C01
:104FB000694C713201508C609D38D140F5405D3CA8
:104FC000F540E140693CB05E2140694C9B6556F676
:104FD000332627DAFAE7BA2550BAAB6546882D564C
:104FE000390C390C390C7BB928F0AE53DD4CF0F09C
:104FF000B023DD4C4E68B8E61F30FE991C590209FB
:105000001C4E702868A87030E69329407118EE3A5B
:1050100046232940F83902690CE34E9902B05D40FD
:10502000DB3550E6672550440CA70C9F2D2C84BB24
:10503000CC3381008C170B6E212C6EBD220484E9C9
:105040004CE667EED704750235500C570CCF088438
:10505000E609231D1E7D2C846B842908E00D54462F
:105060001C1066FB811C590248A0DD4CD91CD84E8F
:1050700070D828E6F62B9A26E3FA46BEBA0E666882
:105080009C0A254CD91CD84E70D8A8294CFA1F4E22
:10509000224C17BEAE381940280E78BE1E1940AEFD
:1050A000DD4CAE684E70B80E384C2793550C154049
:1050B000BE77FE6F23550C4EEE3B43550C1540FE5C
:1050C0007D2C5502550C4EEEC7CB355288091CC1BC
:1050D0004CB0280ED14CF84C1778990C0D40C14CAF
:1050E000389D38D14C384C17B8990C0140C14C4C04
:1050F0001F48030EB02138990CD14C7801400E6244
:10510000990CD14C0D40BD4CB0E8AE9902091C4938
:105110000CF8AEFA271C514E593C3940490C78AE78
:10512000593C3902091C44D14C2EFAAEFD40D14005
:105130004C27A9401B45408D4C35409D4C7D4C4C27
:1051400027284823394038DB091CE50E091CB10C1F
:1051500093091CD14C78EEF84140EE3B0CCF48BB94
:105160008CDF4806B0551C1C6263EADCE3E68C1F4A
:10517000449B0C8783A214FFD4274C177ED4D48E73
:10518000AAEE3CDCCABCAEEE5C1EA05A870EAE6E28
:105190004B8C1B0C9FFA6502BE44F0DB428FA6FAD3
:1051A000E326935CEA8EB0A09C1D4086061CD62B9D
:1051B0008A838A06AEFCAE261C5E2FA6EE8ADBA68C
:1051C0006E11445439029B9CA2A2A2D384488CD76E
:1051D000611C442E5C22029CD84670F8AAA6E8A660
:1051E000AAD86A085A0F046AF3FA13EEDCD0EE3E2E
:1051F000B30CA72E1B0E03C94AAD46AD4A0E51484B
:1052000084B02938094E0EBE77E1407B3540638D6E
:10521000402B550C66662E7A58463E5ED8065E13C5
:105220009E0ED8DCDC8E132E62F354CB98AE5898C9
:10523000FE1B66CEAE5C4ABFEEAE5C0EE66B3A5B22
:10524000C62622DE6EFA604E1EE0C6C36E63424F73
:1052500066EAE32EFAAE4ED84E5C50EEAED8AE4BB8
:10526000FA4B8D402E7A58463EFAEBD8465E139E96
:10527000D85EAE6E2E2BD8EE66D85C4E13228EF31F
:105280002EEED4D4D3AE98A93AAD484E585148EE3C
:10529000C3550CA10C1940386666005BBE008D40FA
:1052A00019422EFAAE5E239C514E3ECEEEB13A6EBE
:1052B000EEEE0EEE5A0EEEE613BA4E9C4217AE8E8E
:1052C0004E6EDC50CE4B22CEF34EEE940FD4CAC3BA
:1052D000C848D1186916C848C8D1189512D11855B0
:1052E00016D118C1120E7118EEB02938AD00613E0A
:1052F0000EAD0021387118693E88FAA00E8E262660
:10530000065C4647D4941BCEE066D34EDA8C93DC21
:10531000D42309102BDC0910D4D409100ECE7D3A09
:105320000E0110DCD417DC0110EE4EEE93883144F0
:105330008C9D3A98D44AB13A5EE05E33DC101BDCB7
:10534000501EF8FCD88404D83C601EE85902214065
:105350001B19401144F05CE0B04C605311440E4CFA
:1053600027B05D40AE584E7078A84E7038689828C7
:10537000E0EE4E70380E7828B868D3BE0021401B8E
:10538000A9404E7078A83868CEBE1E28F8BA9CEAAC
:10539000EAEABAE8AA8A8A8AE071404E70EED8F842
:1053A0001A9ABABABA1CEAE6E838EE7828B868BAA7
:1053B000463CFED8EEE04E7038BE5CEA28F89CEA27
:1053C000EAEAAAA6E8834E70389C534E70781C2BEC
:1053D0004E70B89CEED8F8D4CE14EBFEAED8E0D127
:1053E0004CF8E138D140490C38D3D14C78AEF8E5CF
:1053F00038D140D14CAE7863D14C78E138D140D12E
:105400004CAEB8213835408BE140EB4E1B4EBE5CB4
:10541000502BAEBE2E7A58463E5ED81CD4763654FB
:10542000E3EEEE6BD86EEE4B2687D86E26DFAED855
:105430000E23D8AE2BD8AED86E9E5E5B8E1E263B5A
:10544000D8FCD86EA66E264B66CEBE1ED4D4C34EF4
:10545000AE98EE2E767676007D3A2EFAAEDCCED879
:105460006ECEF66026E63B66EE1ED44ECF66E0A614
:1054700043653EFEEFF6DF0E8E1CEE8A5C4A8F66B9
:10548000061B36E04E22CE3EEEC21BAA260EC223DB
:10549000EE2EFBDE338A6E262EFB6A626B7E5BEE9F
:1054A000865A5E2A4EBAE04E1C985CD476F3CEEE55
:1054B000B00ED6875653DCD42766E3434E4BD41444
:1054C00037A6E38A3A5B1E7E06A61666D3268ED4DE
:1054D0000AA3FA174EA05CF62B86F61F86E0F61F8D
:1054E0004E2B4A6A56D4D4E0BE6E8E588E4E279804
:1054F0000EE026CB5C626E993E2EFAAE84045E13FB
:10550000081E1A6ECEE673CE5E7FDCD494214B2645
:10551000DB8D48C351485C336E66AE333A8EF32E52
:10552000EE66539CE22B62E24F225C43AEFAAEE29F
:105530006B4E5C6A0E1C500C13A66E0E4C3BD14099
:10554000FD40A1408C1BBE1EF93A228EF32E54471B
:10555000EE66D4EE0D46EE4C2BBD48AE6EDC909C54
:10556000FA83DCE22B628E587B268E7EA3463C6259
:105570006E0E0C213D3BAE7EF32E7E983B588EEE98
:10558000EEEE0E6ECEEE2798AEE066CB8ED8268974
:105590003E6E5A5E0E0C1B69444C1BD140F540D93F
:1055A00046EE5C90D010905010501050905050101B
:1055B0000B4E54977A103AD4DF5437147F94BF546B
:1055C000E79CD05C6B9050D05010D0501010509091
:1055D0005CEEE0D0501050D050101010D0D09C9302
:1055E0001CD0D0101050D03068DC3B5CD0D0D01034
:1055F00010D0505CEB5CD0D030311CB330339C9376
:105600002EFAAED14084C14C0EB05EBB06BAF63362
:10561000653EE6EB66EE5ADFE64FBE1EFEFE1EFE60
:105620001388C14C5E6D488D422EFAAE48DA7F3544
:1056300040FAF398FEDF2EF93A2EFAAE44043E5EAD
:1056400087DA73A606E67B461BA6080E5E5A5C8ABE
:1056500062228E588B5CCE62AE4EE94E422766EED9
:10566000E3D8993C8BF540B344043EAE0E26E6B336
:105670005E57AE6D445C4EA60E6E3B08CB54F7D41D
:105680003E26DB7B8E7EF3982EBE3B3E6EEED494A0
:105690009BAE8EEAEAEAAE9CD086C6E35C8EEE8DC7
:1056A00048414CFAE3D4BB2E9C822E8E4D480C37D9
:1056B0006E8E6E2E6E1C414CFA3B8EDBEEDB8E2323
:1056C0005EEF665E0C1BBE009D384CCB354031381A
:1056D00098FEBD46A6EEDB8EBD486E5C1B2E62F3C7
:1056E0004226DCE08CA04ED85148EE693E5E475D14
:1056F0003ED14C5846FA1D36693EF540E30E4E70D9
:1057000038E030E0DB30FDC3B80EF8CEBECECE764A
:105710001356E8AEA8AEE066665C4227FAA6E3AE92
:10572000E01C4E0404C4606E2ED436D4EB1C909062
:10573000901090BCAE1C1D544C29038C2F0C609112
:105740000C4E70606E28F83051A6E8600000EE4BF9
:10575000F643A6300586061388B0E0F6FFD91C0E86
:10576000B0CEFE2F4E8F95464E375C4A2236E0E68D
:105770005B66E6434EE0E62366E687612C0EB019D1
:1057800040F540D140ED384E5090262938D1404E5A
:105790005C2650502140A92C1050353C4E26D0108C
:1057A000D010102140E940A92C50D0353C4E269015
:1057B00050D05050BD40F5404E5CD02938DD404EB1
:1057C000BED84E101010353C4E10662141E940B154
:1057D0004C4E66D84E50501050D01050D0D0901033
:1057E000D02940F540A10C2940A140F5404EBE66AD
:1057F0005C50BD400940B948F938DD40B944D1405A
:10580000612C2EFA0ED140DA5BB02140B14CA140A0
:10581000FD409BF540F93A30FEC54E30FFE38C3138
:1058200032600CD7DC501C62335427DC7ED34C3BF7
:105830007E37A2D4442BBE025437B0C53A069C4AE8
:105840004704C14CF80A65025C4A279C02138A5D32
:105850003AFE2F31444EA0653E811C0D54C14C0DC3
:1058600054B0550C1C428F1540FE6F680EB0288C4A
:105870004F1540FE2B7828B068C14C5CEE1F5033AA
:105880004E50280E781940D14078BD4C6EA32E7A28
:10589000F540680EB819408C2778613CF938F63726
:1058A0003BE140F9388D422940A02550FA5C505028
:1058B000D010D05090909050237AFA7ADC133A624C
:1058C000F354BB19483AB8BAA8BA4E669D393902A2
:1058D00060E61686662550E6952A58F8E61F30FCE5
:1058E0000698DCD01C6A1F883C3EFEA6065670381F
:1058F0001E7EB6561B3CDB6A6A8B3C7E3EDF668CA6
:10590000334CB74884CB1676A6C3BEBCF666844437
:10591000E05CC44813448460795C4E70E0AE28FEBD
:105920001BFE4F0C3B9CE21FD013D0A83C364F45CA
:105930000CD61B5C903C4EB83C365F450CD61B9C8D
:10594000107CEEEE4EB83C364F450CD61B1C103C7E
:105950004EB87C364F450CD61B9C10FC4EB8BC365E
:1059600057450CD61390FCEEEE4EAE755C0EB87C2F
:10597000365F450CD61B5C90BCEEEE4EB8BC364F85
:10598000450CD61B5C90BC4EB83C365F450CD61B14
:105990009C103CEEEE4EB87C365F450CD61B5C107E
:1059A0007CEEEE4EB8FC364F450CD61B9C10FC4EE0
:1059B000AE615C8C234C3D5FF8FE434E3008A8304E
:1059C0000C3B4E300CA8300868A0381E7E877E57EE
:1059D0007E73B8BCEEEE4E7C1B787C4E6E815AA076
:1059E000BE600EFC9C02788C234C174EA297A20F2F
:1059F000A25FA27FA2F7A25FA27FA2F7A2477B7C51
:105A00004EB87CEEEE4E6EB87CEEEE4EB8BC4EC399
:105A10007C4EB8BCEEEE4E6EB83C4E637CEEEE4E65
:105A20006EB87C4EB8BC4E9CB0FE23109C42787081
:105A3000686E6D5C8C1B4C37F85A46FEFE3B1C10A2
:105A4000FE1B1C105EDC8C1350695C4E5C0C13500A
:105A50001CCC1B223BA0D423E01C50555C38EEA08C
:105A6000E020E00E7870682B0EB870A88C2BCCA0CC
:105A700048E04C60C8CC60889D0EA01C109C502053
:105A80001378EE68A886910C4E5C906EF7CCEB30E4
:105A900026065ABC3006203C5666876E66302806BD
:105AA0000F4E9C9090683CA89D02664EA02660A672
:105AB000E33C4B4E26263C234EE34E5CF0514E8198
:105AC0001CB02844D95C6ECD00AEF0986E5FA01C6F
:105AD000100626E630187CBA233A7A333046DB26A5
:105AE000CB86468748D95C6EB0CE4E3A30F3A66E70
:105AF00047CD000E986E174E7038704E6E68A8CC69
:105B0000A0848102A0CD00F0F0D8D8D8D8D8D8EEA3
:105B10006ECD00CE4EB15F584E300770EE384EAEAF
:105B20004CA72EAED8F04E38D8F030E0AEEE66A0DE
:105B30006E664B563B8E00630920F8E637300CE862
:105B4000E6E6C8CC2366E3E09D0CCD4E00000304DE
:105B5000050A08060BFF0209070D010C00FF2020B3
:105B600020205F5F7C002C0044697370206F6666A4
:105B70000D0A00555345520046004700424547492B
:105B80004E0052414400442E4D59005052474D00A2
:105B90005553455220202000662020006720200019
:105BA000424547494E2020202020005241442020D9
:0F5BB0002000442E4D59202020004320202000AB
:105BBF00883C000000000000050D0000A03C000024
:105BCF00A53C0000A33C0000FF0000005D060000A4
:105BDF00AF3C0000B93C0000473C00000000000053
:105BEF0049040000CB3C0000A53C0000D73C00005E
:105BFF000000000055050000D93C0000A53C000046
:105C0F00E53C000000000000B5060000E73C000086
:105C1F00A53C00000F000000F40100000401030187
:105C2F000201010411040F041704160118010000EA
:105C3F00905B0000985B00009C5B0000A05B000085
:105C4F007A5B0000AB5B0000B25B0000BA5B000048
:105C5F008B5B000000171B243E425369750502053C
:105C6F000804080B080404050105040908090406C3
:105C7F0008070206020402060106040701030803CF
:105C8F00040C080D020C0203020C010C040D010D93
:105C9F00080D040802080807080202070408010893
:105CAF0004090209010A080B020A0201080A010A83
:105CBF00040B01020802041008110210021108104F
:105CCF000110041101120212011302130812080F1E
:105CDF0008120413011304140214011502150814F9
:105CEF000817081404150115041702170119081ACB
:105CFF000219021602190119041A01160816041BBB
:105D0F00021B081A0818021A041B011B0418081892
:105D1F00040B042020202020202020202000000021
:105D2F0001000000735B0000785B00007A5B0000ED
:105D3F007C5B00007A5B0000825B0000865B0000EA
:085D4F000B3600008B5B000025
:04000003000033BD09
:00000001FF
